:100000000C945D020C94AF020C94AF020C94AF02FE
:100010000C94AF020C94AF020C94AF020C94AF029C
:100020000C94AF020C94AF020C94AB1E0C947D1F89
:100030000C943D2D0C94AF020C94AF020C94AF02C3
:100040000C94AF020C94AF020C94AF020C94AF026C
:100050000C94AF020C94620B0C94AF020C94AF02A0
:100060000C94AF020C94AF020C94AF020C94AF024C
:100070000C94AF020C94AF020C94AF020C94AF023C
:100080000C94AF020C94AF020C94AF020C94AF022C
:100090000C94AF020C94AF020C94AF020C94AF021C
:1000A0000C94AF020C94AF020C94AF02EA1F0C2028
:1000B000FA200C20FA2051207420FA20C920DC20DC
:1000C000C023C023EF23EF234D248B24A526A52690
:1000D000A424A526A525A5257926A526A52690260E
:1000E000808080800405060708090A0B0C0D0E0F9E
:1000F000101112131415161718191A1B1C1D1E1F88
:10010000202122232425262728292A2B2C2D2E2F77
:10011000303132333435363738393A3B3C3D3E3F67
:10012000404142434445464748494A4B4C4D4E4F57
:10013000505152535455565758595A5B5C5D5E5F47
:10014000606162636465666768696A6B6C6D6E6F37
:100150007071727380808080808080808080800356
:100160000201808080808075007476778080808036
:10017000808080808080808080808080808080807F
:10018000808080808080808080808080808080806F
:10019000808080808080808080808080808080805F
:1001A000808080808080808080808080808080804F
:1001B000808080808080808080808080808080803F
:1001C00078797A7B7C7D7E7F808080808080808053
:1001D000808080808080808080808080808080801F
:1001E0000A00253031366200253032643A20000A98
:1001F000722F63203031323334353637383941424B
:10020000434445460A0073706565643A2025730AC5
:10021000007573625F73746174653A2025303258DB
:100220000A00686F73742E5461736B3A2025640A58
:10023000000D0A0020253032580073746174653A4D
:100240002020253032582025303258000D0A002059
:100250002530325800696E7075742025643A20206C
:10026000253032582025303258005B445D005B4316
:100270005D003C03550053004200200074006F00F5
:10028000200055005300420020006B0065007900FB
:1002900062006F00610072006400200063006F0064
:1002A0006E00760065007200740065007200000048
:1002B0000E0374002E006D002E006B002E00000057
:1002C0000403090409027400040100A032090400B7
:1002D0000001030101000921110100012240000772
:1002E00005810308000A0904010001030102000955
:1002F0002111010001224D000705820308000A09AF
:10030000040200010300000009211101000122364E
:10031000000705830308000A090403000203000024
:100320000009211101000122220007058403200099
:10033000010705040320000112011001000000085C
:10034000EDFE5B001408010200010631FF0974A1F3
:10035000010975150026FF009520750881020976B0
:10036000150026FF00952075089102C0050109803F
:10037000A101850216810026B7001A81002AB70064
:10038000751095018100C0050C0901A101850316B6
:100390000100269C021A01002A9C02751095018119
:1003A00000C005010902A1010901A1000509190107
:1003B0002905150025019505750181029501750333
:1003C00081010501093009311581257F95027508E4
:1003D000810609381581257F950175088106050C70
:1003E0000A38021581257F950175088106C0C00570
:1003F000010906A101050719E029E7150025019566
:100400000875018102950175088101050819012906
:10041000059505750191029501750391010507196F
:100420000029FF150026FF00950675088100C063AE
:100430006F6E73756D65723A20253034580A0073FB
:10044000797374656D3A20253034580A000A002506
:1004500030325820006B6579626F6172643A200017
:100460004C45443A20253032580A00290A002575A7
:10047000002F002575005D280025640020002564FC
:1004800000200025640020002564007C0025303217
:1004900058006D6F7573656B6579205B62746E7C57
:1004A000782079207620685D287265702F61636CF2
:1004B000293A205B0000D009B60A11241FBECFEFF5
:1004C000DAE0DEBFCDBF04B603FE27C080918B0407
:1004D00090918C04A0918D04B0918E048730904B44
:1004E000A740B04BD1F410928B0410928C04109260
:1004F0008D0410928E0414BE84B7877F84BF0FB61C
:10050000F894A895809160008861809360001092B3
:1005100060000FBEE0E0F8E3099511E0A0E0B1E073
:10052000E4EDF3E602C005900D92A839B107D9F7C2
:1005300024E0A8E9B1E001C01D92AB38B207E1F7B1
:1005400012E0CDE5D2E004C02197FE010E94CE3139
:10055000CB35D107C9F70E940B0A0C94E8310C94F3
:100560000000FF93EF93E0919801F091990130978B
:1005700009F00995EF91FF910895FC018591803074
:1005800011F0EFDFFBCF0895FF27E0E230E247FFF5
:100590000CC0419597FF09C0EDE26095709580957C
:1005A0009095611D711D811D911D27FF02C0219530
:1005B00030E350E2AA27660F771F881F991FAA1FF2
:1005C000A41710F0A41B63955A95A9F7AA3008F058
:1005D000A95FA05DAF93F395611571058105910544
:1005E00041F7ED3211F4EF93F395F21718F43F93BE
:1005F000F395FBCF8F91B5DFFA95E1F70895E99177
:10060000F9918591803021F0853219F0AADFF9CF78
:10061000089520E0E89455915532C1F3503311F418
:10062000689455915A3348F4505390F3220F022E98
:10063000220F220F200D250FF4CF0EF42195899162
:100640009991533619F3533729F1533559F1BC01B8
:1006500088279927E8945C3621F4899199916894C8
:100660005591543639F446EF7EF077FF0DC08FEF89
:100670009FEF0AC055374AE039F0583540E121F084
:10068000523642E009F00895FF93EF937DDFEF913A
:10069000FF91B7CFFF93EF93FC0181918030B9F3C5
:1006A00060DFFBCFFF93EF9368DFF1CFDF93CF9352
:1006B000CDB7DEB72596A3DFCF91DF91089580E017
:1006C0000895089580E0089581E00895CF93DF9321
:1006D000CDB7DEB728970FB6F894DEBF0FBECDBFFB
:1006E00029833A834B835C836D837E838F839887D2
:1006F0008091D202282B2093D202FE013396AE01C4
:10070000475F5F4F2191243088F080E090E0DC016A
:10071000AE52BD4F12963C911297311103C0129602
:100720002C9304C001968630910589F7E417F507EC
:1007300049F728960FB6F894DEBF0FBECDBFDF9104
:10074000CF910895860F911D860F911DFC0156874C
:10075000458781E00895CF93DF93EC018C819D81E3
:10076000DC01ED91FC910480F581E02D6E8109950D
:100770001F86188A81E08A8B1E821B8A1C8A1D8A2A
:100780001E8A1F8A80E0DF91CF910895FC01868147
:10079000089581E0633009F080E0089581E06130E0
:1007A00009F080E00895860F911D860F911DFC01D0
:1007B000858596850895FC0187890895EF92FF92BB
:1007C000CF93DF93DC01E70152968C9152978230F0
:1007D00049F11F966C931F9750964C9350979B81AD
:1007E00093709330F9F49A8197FF1CC09E815896BC
:1007F0002C915897291718F458969C935897E82FDE
:10080000F0E09F01220F331FE20FF31FEA0FFB1FDF
:100810009A819F7097839C81908794E091878F5FE6
:1008200052968C93DF91CF91FF90EF900895EF92C5
:10083000FF920F9302970E94DE030F91FF90EF90BB
:1008400008950895DF92EF92FF920F931F93CF9335
:10085000DF93CDB7DEB762970FB6F894DEBF0FBE59
:10086000CDBFDC0157962C91222381F07C010E94A0
:10087000C70AF7010389148925893689DC01CB0170
:10088000801B910BA20BB30BB7FF02C0D12C39C058
:10089000838590E09A8B898B8E010F5F1F4F9E019D
:1008A0002F5E3F4F42856681848195810E94CC13E3
:1008B000D82E811118C029893A892330310598F042
:1008C000D7011D968D919C911E97009761F0DC01D8
:1008D000ED91FC910190F081E02D8E010F5F1F4F93
:1008E00040E0B70109950E94C70AF701208DDC019D
:1008F000CB01820F911DA11DB11D838B948BA58B04
:10090000B68B8D2D62960FB6F894DEBF0FBECDBFAD
:10091000DF91CF911F910F91FF90EF90DF9008959D
:100920003F924F925F926F927F928F929F92AF927F
:10093000BF92CF92DF92EF92FF920F931F93CF93CC
:10094000DF93CDB7DEB7EC970FB6F894DEBF0FBEDE
:10095000CDBFDC0114968D909C90159716963C9116
:10096000311139C1522E342E462E5C01FC01108EFD
:10097000D401ED91FC910190F081E02D60E0C40183
:1009800009957C01009711F486ED2AC1FC01608075
:1009900071806114710409F420C16501F7E0CF0E84
:1009A000D11CDC011196DC92CE9214965C928E01E1
:1009B000065D1F4F28E030E040E060E0F5018481F3
:1009C00095810E948F118CAF8111F8C01AA5D701B3
:1009D0006D927C92D401ED91FC910280F381E02D27
:1009E000232D40E0642DC4010995F50186838823F9
:1009F00009F4F5C099A99087282F40E060E0848130
:100A000095810E943A128CAFD401ED91FC91D701EF
:100A100014961C92882359F00480F581E02DD501AD
:100A200016966C91C4010995F5011682D2C0019009
:100A3000F081E02DD50116966C91C4010995FC0159
:100A4000892B09F4A1CF912F133108F092E1548240
:100A5000992369F0292F30E08E01065D1F4F40E099
:100A6000F5016681848195810E948F118CAF8CADD8
:100A70008111A7C0EBACF12C40E2642E41E0742E52
:100A80002501F2E04F0E511C4E0181E1880E911CB0
:100A9000FE1449F17A8269825C824B821E86188A32
:100AA0001F8619A21AA21BA219A69F828E8299865E
:100AB00088868D818B878A879D868C868E010F5FC5
:100AC0001F4F2F2D40E0D50116966C911697149666
:100AD0008D919C9115970E94DD11F50182898230DC
:100AE00011F0F394D5CFD50152968C91823019F044
:100AF00081ED8CAF66C0960142E0F501668184818C
:100B000095810E94C90C8CAF68EE73E080E090E0A4
:100B10000E94C90AD5011F962C911F9740E0169696
:100B20006C91169714968D919C9115970E94A7131E
:100B30008CAF811146C068EE73E080E090E00E94C7
:100B4000C90A40E060E0C5010E949D158CAF81118B
:100B500038C020E040E060E0C5010E9473158CAF12
:100B600086E291E09A838983AE014F5F5F4F60E038
:100B700070E0C5010E94021580E28CAF8CAD882325
:100B8000C1F090E0959587958CAFFE01FC966F01C2
:100B9000EE24E394F12C00E022E040E060E0C501A7
:100BA0000E94451569E170E080E090E00E94C90A6A
:100BB000E5CF91E0D50157969C9312C0F701718261
:100BC0006082D501ED91FC910480F581E02DC50195
:100BD00009958CAD05C089ED03C087ED01C084ED9A
:100BE000EC960FB6F894DEBF0FBECDBFDF91CF916C
:100BF0001F910F91FF90EF90DF90CF90BF90AF903B
:100C00009F908F907F906F905F904F903F9008954E
:100C10000F931F93CF93DF936091D2017091D30113
:100C2000E091A101F091A2014091C6015091C7014C
:100C30002091BA013091BB018091AE019091AF013A
:100C40006E177F07B1F4E0919F01F091A0014E175C
:100C50005F0779F4E0919D01F0919E012E173F0707
:100C600041F4E0919B01F0919C018E179F0709F4DC
:100C70009DC07093A2016093A1015093A001409385
:100C80009F0130939E0120939D0190939C0180933E
:100C90009B01E2EDF2E088E0DF011D928A95E9F721
:100CA0002091CA013091CB014091CC015091CD01EE
:100CB0006091CE017091CF018091D0019091D101CE
:100CC0000E9466032091BE013091BF014091C00196
:100CD0005091C1016091C2017091C3018091C40122
:100CE0009091C5010E9466032091B2013091B30139
:100CF0004091B4015091B5016091B6017091B70176
:100D00008091B8019091B9010E9466032091A601DB
:100D10003091A7014091A8015091A9016091AA01C9
:100D20007091AB018091AC019091AD010E9466037E
:100D300081E08093D1028091730480FF14C0809180
:100D4000D3021F928F938091D2021F928F938AE3D6
:100D500092E09F938F930E9456030F900F900F90F5
:100D60000F900F900F90C0E0D0E004E312E080916C
:100D7000730480FF0EC0FE01EE52FD4F82811F9270
:100D80008F931F930F930E9456030F900F900F9015
:100D90000F902196C630D10551F78091730480FFE2
:100DA00007C081E392E00E94BD0202C01092D1020E
:100DB0000E94200BEC018AE592E00E940314CE0110
:100DC0000E94380B8536910580F02091730420FF36
:100DD0000CC09F938F9382E292E09F938F930E9427
:100DE00056030F900F900F900F90C0919A018AE5D3
:100DF00092E00E94A20CC817B9F18AE592E00E9425
:100E0000A20C80939A019091730490FF0CC01F92E2
:100E10008F9381E192E09F938F930E9456030F90EE
:100E20000F900F900F9080919A018039E9F4809192
:100E3000730480FF15C08091A301823019F088E10E
:100E400091E002C083E191E09F938F9386E092E06E
:100E50009F938F930E9456030F900F900F900F90C7
:100E60000E9417210E94A22281E0DF91CF911F9161
:100E70000F910895482F50E0CA0124E0880F991F70
:100E80002A95E1F7805E9109089730F48091D202AB
:100E9000882311F090E002C080E090E0E4EDF2E001
:100EA000A1E0B0E036E03E0F2191243080F0622FC7
:100EB00062956F7070E04617570749F42F70BD01B7
:100EC00002C0660F771F2A95E2F7862B972B3E13F9
:100ED000EBCF0895EF92FF920F931F93CF93DF9381
:100EE0008FEE91E00E94BD02C0E0D0E088EEE82ED7
:100EF00081E0F82E02EE11E0DF93CF93FF92EF92A4
:100F00000E9456038C2F0E943A070E940B2D9F933C
:100F10008F931F930F930E94560380EE91E00E94DF
:100F2000BD0221968DB79EB708960FB6F8949EBF66
:100F30000FBE8DBFC031D105F9F6DF91CF911F9162
:100F40000F91FF90EF900895CF92DF92EF92FF9272
:100F50000F93CF93DF931F92CDB7DEB78983CE0176
:100F600001966C01EE24E394F12C00E022E040E0D5
:100F700060E08FE192E00E94451522E040E060E0F1
:100F800086E092E00E94451522E040E060E08DEEB0
:100F900091E00E94451522E040E060E084ED91E0A0
:100FA0000E9445150F90DF91CF910F91FF90EF9028
:100FB000DF90CF900895FC01758364838CE291E00B
:100FC000918380838AE491E093838283138A148AD5
:100FD000158A168A178A178288E080878CE38187B2
:100FE0001286138684E0848781E0828B118A1786BB
:100FF0001686158661157105B1F0DB01AA5ABF4F3F
:1010000080E090E02D913D91232B49F48B96880F41
:10101000991FDB01A80FB91FED93FC93089501966A
:101020008031910579F708952E9A08952E988EBDF6
:101030000DB407FEFDCF1EBC0DB407FEFDCF0E9410
:1010400014088EB508952E9882608EBD0DB407FEEB
:10105000FDCF6EBD0DB407FEFDCF0C94140888EFD4
:101060000E941608807C8034A1F018F4882301F1D6
:101070000895803819F0803CB9F0089588ED0E94F9
:10108000160881FD0BC069EC88ED0E94230882E000
:101090000CC088ED0E94160881FDF5CF6BEC88ED41
:1010A0000E94230883E001C081E08093A30108959A
:1010B00061ED88ED0E9423081092A30108950F931B
:1010C0001F93CF93DF938C01269A0E941408219AD4
:1010D000229A2398209A80E58CBD81E08DBD2598C9
:1010E00068E188E80E94230860E288E70E942308FC
:1010F00060E088E70E942308C1E0D0E0209799F0E3
:1011000088E60E941608219680FFF8CF61EC88EDF2
:101110000E94230860E680ED0E94230864E088EEC8
:101120000E94230802C08FEF11C088EE0E941608AB
:1011300082FFFBCFC8010E942F0860E288EC0E946A
:10114000230861E080E80E94230880E0DF91CF91CE
:101150001F910F9108958AE592E00E945F0888EC44
:1011600091E090932D0280932C028CEB91E0909370
:1011700014028093130280EB91E09093FB01809323
:10118000FA0184EA91E09093E2018093E1010895ED
:10119000EF92FF920F931F93CF93DF93EC017B01AC
:1011A0008A0188A1823029F128F4882341F0813016
:1011B00081F0C9C0833019F18430D9F1C4C082E014
:1011C0008C832D813E8138872F838A87898781E0B0
:1011D00088A3A801B701CE0107960E948F1981113B
:1011E00002C080E0B1C0ED81FE81808189A3818150
:1011F0008AA3CE0142969E838D8383E088A38AA131
:10120000843059F018F4823049F00AC0853039F042
:10121000813231F489A1825002C01BA287E08C8305
:101220008D819E8198878F838C818A87898784E0CE
:1012300088A38AA1843081F0853091F1823009F051
:1012400050C0A801B701CE0107960E948F198823CC
:1012500041F28D898CA372C0A801B701CE01079617
:101260000E948F19882309F4BCCF8D89833009F03F
:1012700065C08E89813009F061C098A58F89992356
:1012800021F0882309F45AC003C0813009F056C008
:1012900091E09BA39A899EA39B899FA38DA34EC097
:1012A000A801B701CE0107960E948F19882309F47F
:1012B00098CF8BA1882309F441C08A819B81009734
:1012C000E9F1DC01ED91FC910190F081E02D7E01CE
:1012D000B0E1EB0EF11C0DA12FA14EA16CA109955F
:1012E0002DC089A19D85992319F09130E9F021C085
:1012F00090E002979F878E8781E08D8715C0F80167
:1013000020813181232BA9F001979F878E87F701D8
:1013100080819181019691838083D8018D919C91E8
:10132000119701978D939C938E859F85009739F730
:101330001D868E859F85892B09F053CFCE0140965F
:101340009E838D8318A281E0DF91CF911F910F9131
:10135000FF90EF9008950F931F93CF93DF9300D0EA
:1013600000D0CDB7DEB78C017C836B835A83498371
:101370002B813C81232B59F0AE014D5F5F4FBE01A5
:101380006F5F7F4FC8010E94C8088111F1CF0F9095
:101390000F900F900F90DF91CF911F910F910895B3
:1013A0008AE592E00E94710C6AE572E089E492E0BD
:1013B0000E9422186AE572E088E392E00E942218F7
:1013C0006AE572E08FE192E00E94DB076AE572E075
:1013D00086E092E00E94DB076AE572E08DEE91E024
:1013E0000E94DB076AE572E084ED91E00E94DB0772
:1013F00080E591E09093C9018093C8019093BD016D
:101400008093BC019093B1018093B0019093A501AA
:101410008093A4010895569A5E9A80917304816026
:1014200084608093730480E091E00E94122184B76D
:10143000877F84BF0FB6F894A8958091600088617B
:1014400080936000109260000FBE90E080E80FB6BD
:10145000F89480936100909361000FBE0E94301E4B
:101460000E948D1E8091E20084608093E2008EEEE7
:1014700099E10E94F02C0E94D32178940E94D721F8
:10148000FDCFEF92FF920F931F93CF93DF93EC0169
:101490007B01DC01129688E0F80101900D928A959B
:1014A000E1F70E94C70A7B876A878091730480FFF7
:1014B0001EC00B811A81D701ED91FC910084F1854A
:1014C000E02DC70109951F920F931F921F931F9242
:1014D0008F9385E592E09F938F930E9456038DB77B
:1014E0009EB708960FB6F8949EBF0FBE8DBF249688
:1014F00016E08FE4E82E82E0F82E8091730480FFDE
:101500000BC088811F928F93FF92EF920E94560327
:101510000F900F900F900F90115021961111EDCF59
:101520008091730480FF0AC08CE492E0DF91CF9138
:101530001F910F91FF90EF900C94BD02DF91CF911E
:101540001F910F91FF90EF900895089580E090E033
:1015500008958FEF9FEF08958FEF9FEF08950895FF
:10156000862F0E94EE1981E090E00895EAEDF2E006
:101570001382128288EE93E0A0E0B0E0848395832A
:10158000A683B78386E591E09183808308950C94C8
:101590002C0B8F929F92AF92BF92CF92DF92EF92DD
:1015A000FF920E948A304B015C0120E030E04AE764
:1015B00055E40E9441316B017C0120E030E040E8BD
:1015C0005FE30E944F3087FD24C020E03FEF4FE7EC
:1015D00057E4C701B6010E943C311816ACF420E074
:1015E00030E040E251E4C501B4010E9441310E9463
:1015F0005B3020E931E06115710581F0C901019787
:10160000F1F761507109F7CFC701B6010E945B3055
:1016100002C061E070E0CB010197F1F7FF90EF901D
:10162000DF90CF90BF90AF909F908F90089582E011
:1016300084BD93E095BD9AEF97BD80936E000895A9
:101640002FB7F8948091E8029091E902A091EA0204
:10165000B091EB022FBF08952FB7F8946091E80284
:101660007091E9028091EA029091EB022FBF0895F8
:10167000CF92DF92EF92FF920F931F932FB7F894C0
:101680004091E8025091E9026091EA027091EB0208
:101690002FBF6A017B01EE24FF248C0120E030E0A3
:1016A000C016D106E206F30610F4415051099A0122
:1016B000281B390BC9011F910F91FF90EF90DF900C
:1016C000CF9008951F920F920FB60F9211248F930F
:1016D0009F93AF93BF938091E8029091E902A0910C
:1016E000EA02B091EB020196A11DB11D8093E802C0
:1016F0009093E902A093EA02B093EB02BF91AF91FD
:101700009F918F910F900FBE0F901F901895CF93C0
:10171000DF93FC01862F807809F051C0283008F053
:101720004FC0442321F09581973009F449C0EF015F
:101730002D96A0E0B0E011969881911103C0662328
:1017400031F021C02596AF30B105A9F739C085E049
:101750008A9FE0018B9FD00D1124CE0FDF1F442301
:1017600031F081E4888785818F5F858302C081E0C5
:10177000888725E02A9FC0012B9F900D1124E80F38
:10178000F91F80851DC06770660F660F660F4423C2
:1017900041F0606485818F5F85838770687F682BE7
:1017A00003C02770687B622B25E02A9FC0012B9F16
:1017B000900D1124E80FF91F6087862F01C080E08B
:1017C000DF91CF910895DF92EF92FF920F931F93D5
:1017D000CF93DF93EC01E62EF12C85E0689FB001FA
:1017E0001124FE01E60FF71F8085182F177086FF62
:1017F00021C001E085E0D82E8FEF800F8F3008F0F8
:1018000001E0FE01D09EE00DF11D1124808586953A
:10181000869586958770811305C0602FCE010E9442
:10182000E30BEACF0F5F003161F78D81811302C0B6
:1018300011501D8385E08E9DF0018F9DF00D1124C8
:10184000EC0FFD1F108681E0818712862296D783D8
:10185000C683DF91CF911F910F91FF90EF90DF90A2
:101860000895611102C006960895FC013D9621E09D
:101870003081361307C035E0239F800D911D112460
:10188000069608952F5F3596203191F780E090E01D
:101890000895FC016134C1F43F969C01265A3F4FE4
:1018A00061E0AC014E5F5F4FDF0112971C92119611
:1018B0006C93108213974D935C933596E217F30760
:1018C00099F7FC01158208953D9621E03081361389
:1018D00003C0622F0C94E30B2F5F35962031B1F7D4
:1018E0000895CF93DF93FC0188E691E09183808394
:1018F0001582108681E081871286CF010296978338
:101900008683128228E023832CE32483DF011F9641
:101910009F01265A3F4F41E0ED0122971882219600
:1019200048831C922397998388831596A217B3073F
:1019300099F7EA58FF4F108281E18093F002DF911E
:10194000CF9108958091F0020895CF93DF931F9275
:10195000CDB7DEB749830E94310C4981009789F0E9
:10196000DC01ED91FC911197309759F013969C9101
:1019700080E0891731F02081241731F033968F5F92
:10198000F8CF80E090E001C0CF010F90DF91CF91C0
:1019900008950F931F93CF93DF932115310571F0B5
:1019A000E901042F162F0E94310CFC01892B41F014
:1019B0001283D183C083038380E003C088ED01C01C
:1019C00086EDDF91CF911F910F910895CF92DF9215
:1019D000FF920F931F93CF93DF93662381F1F62E2F
:1019E0008C016C0186E5C80ED11CC0E0D0E0D601A8
:1019F0008D919D916D010097F1F0DC01ED91FC91CD
:101A00000084F185E02D09958F1115C0AB96CC0FA0
:101A1000DD1FC00FD11F88819981DC01ED91FC9100
:101A20000480F581E02DDF91CF911F910F91FF9000
:101A3000DF90CF9009942196C031D105C1F680E0A6
:101A4000DF91CF911F910F91FF90DF90CF9008957C
:101A50002E980895CF93DF931F92CDB7DEB7898379
:101A60000E94280D89818EBD0DB407FEFDCF1EBCDE
:101A70000DB407FEFDCF0E9414088EB50F90DF91C4
:101A8000CF910895CF93DF9300D0CDB7DEB76A83AF
:101A900089830E94280D898182608EBD6A810DB480
:101AA00007FEFDCF6EBD0DB407FEFDCF0F900F906A
:101AB000DF91CF910C9414088F929F92AF92BF92B6
:101AC000DF92EF92FF920F931F93CF93DF931F92BA
:101AD000CDB7DEB74C01D62E590149830E94310C97
:101AE0007C014981009709F440C0FC01808191810B
:101AF000892BE9F16D2DC4010E94A50CF50191839C
:101B000080830097B1F1FC0122812695269530E073
:101B10002031310514F02FE030E081E090E0A0E0CA
:101B2000B0E004C0880F991FAA1FBB1F2A95D2F7E7
:101B30000197F801918380836D2D80EE0E94420D04
:101B400088ED0E942A0D682FF7018481882339F0DF
:101B5000F401EA58FF4F80818260682B01C0697FE1
:101B600088ED0E94420D80E005C086ED03C087ED40
:101B700001C08BED0F90DF91CF911F910F91FF90DE
:101B8000EF90DF90BF90AF909F908F9008958F92CD
:101B90009F92AF92BF92CF92DF92EF92FF920F93FC
:101BA0001F93CF93DF93862E942E59010E94C70A6C
:101BB0006B017C0128E8C20E23E1D21EE11CF11C5E
:101BC00000E010E0D0E0C0E098280E94C70ADC01E5
:101BD000CB018C199D09AE09BF09B7FF2DC0692D36
:101BE00080EF0E94420D0E94C70ADC01CB018C19D4
:101BF0009D09AE09BF09B7FF09C088EC0E942A0DF4
:101C000087FFF1CF60E888EC0E94420D88EF0E94C8
:101C10002A0DC82FCF70C43019F0CE3051F00CC04F
:101C20000F5F1F4FA114B10481F20A151B0569F65D
:101C300003C0DF5FD33049F68C2FDF91CF911F9126
:101C40000F91FF90EF90DF90CF90BF90AF909F905B
:101C50008F9008959F92AF92BF92CF92DF92EF92B2
:101C6000FF920F931F93CF93DF937C01C42F122F0A
:101C7000992493946C01C60ED11CC60ED11C86E526
:101C8000C80ED11CA42EB12CABE2AA0EB11CAA0C1A
:101C9000BB1CAE0CBF1CF60180819181DC01ED9173
:101CA000FC910280F381E02D202F412F6C2F0995AC
:101CB000803EC9F4C1110BC061E088EE0E94420D64
:101CC00066E670E080E090E00E94C90A16C0F50167
:101CD00080819181DC01ED91FC910284F385E02DFE
:101CE000612F09950AC08D3031F49FEF990D933023
:101CF00008F040C016C081113DC0F601808191817D
:101D0000DC01ED91FC910190F081E02D202F412F1D
:101D10006C2F0995D82F8D3061F48FEF890D8330AA
:101D200050F464E670E080E090E00E94C90A939469
:101D3000B2CF8823F1F0C1110BC061E088EE0E94A0
:101D4000420D66E670E080E090E00E94C90A11C092
:101D5000EC2FF0E0BB96EE0FFF1FEE0DFF1D808114
:101D60009181DC01ED91FC910284F385E02D612FDE
:101D700009958D2FDF91CF911F910F91FF90EF90DB
:101D8000DF90CF90BF90AF909F9008950F931F93D7
:101D9000CF93DF9300D0CDB7DEB78A016A83898302
:101DA0000E94280D898182608EBDF8016A81862F8C
:101DB000882339F00DB407FEFDCF91919EBD81506F
:101DC000F7CF060F111D0DB407FEFDCF0E941408BA
:101DD000C8010F900F90DF91CF911F910F9108953F
:101DE0002F923F924F925F926F927F928F929F922B
:101DF000AF92BF92CF92DF92EF92FF920F931F9319
:101E0000CF93DF9300D000D01F92CDB7DEB77D8394
:101E10006C835A016901FB0121808FEF820D8034B0
:101E200008F075C00E94C70A2B013C01F8E84F0E6C
:101E3000F3E15F1E611C711CEC81FD81828180FDDC
:101E400002C060E401C060E888EE0E94420D20E01C
:101E5000312CC114D10409F44AC076012C143D047C
:101E600008F47101EA82A8016E2D80E10E94C60E7D
:101E70006E2D88E30E94420DEC81FD8160816062DD
:101E800080EF0E94420D88EC0E942A0D87FFFBCF55
:101E900060E888EC0E94420D88EF0E942A0D282FEE
:101EA0002F70812C912C1982222361F02B830E94A8
:101EB000C70ADC01CB0184199509A609B7092B8152
:101EC000B7FD05C0CE18DF080E0D1F1DC2CF26308E
:101ED00001F12E3009F456C0243049F4FFEF8F1A77
:101EE0009F0AA114B10459F18A149B0441F588EFAB
:101EF0002B830E942A0D85FB882780F9EC81FD81C8
:101F0000928180FB90F992832B81822F41C08AEDD0
:101F10003FC088EF0E942A0D85FB882780F991E059
:101F20008927EC81FD81928180FB90F9928390FD5D
:101F300002C060E401C060E888EE0E94420D60E0EB
:101F400088E30E94420DF801608180E10E94420D09
:101F50006A8188E30E94420DEC81FD8160816062AC
:101F600080EF0E94420D88EC0E942A0D87FFFBCF74
:101F700060E888EC0E94420D88EF0E942A0D282F0D
:101F80002F7092CF89818F5F89838330C1F6AFCF65
:101F90000F900F900F900F900F90DF91CF911F91A6
:101FA0000F91FF90EF90DF90CF90BF90AF909F90F8
:101FB0008F907F906F905F904F903F902F900895FB
:101FC0002F923F924F925F926F927F928F929F9249
:101FD000AF92BF92CF92DF92EF92FF920F931F9337
:101FE000CF93DF9300D000D01F92CDB7DEB75C0156
:101FF0007D836C834A017901F901C080D180FB01A6
:102000004180F90111821082FB01828181FD02C0B1
:1020100060E101C060E288EE0E94420D3C2C940118
:10202000EC81FD81408160E0C5010E94C70D582E02
:10203000F6E08F1316C088EF0E942A0D82958170FA
:1020400091E08927EC81FD81928180FB91F9928357
:1020500091FD02C060E101C060E288EE0E94420D85
:10206000DECF81115BC088EC0E942A0D82FF54C034
:1020700080E30E942A0D282E282F30E0C216D306B6
:1020800008F4232CF70120813181622C712CA601E8
:10209000421B530B57FF02C040E050E0930146152E
:1020A00057050CF49A0129833A832B830E94280D4B
:1020B000F8E0FEBD8B813A8129810DB407FEFDCF8A
:1020C000F801882341F01EBC81500DB407FEFDCFFE
:1020D0004EB54193F6CF020F131F0E94140864E01F
:1020E00088EC0E94420DF70120813181620E731E3F
:1020F00071826082241420F06C147D0408F48FCF68
:1021000088EF0E942A0D82958170EC81FD81928179
:1021100080FB91F9928302C080EF582E852D0F909D
:102120000F900F900F900F90DF91CF911F910F9113
:10213000FF90EF90DF90CF90BF90AF909F908F90E7
:102140007F906F905F904F903F902F9008952F92C7
:102150003F924F925F926F927F928F929F92AF9237
:10216000BF92CF92DF92EF92FF920F931F93CF9384
:10217000DF93CDB7DEB762970FB6F894DEBF0FBE20
:10218000CDBF3C01542ED22E402E5E2D2FA038A460
:10219000E9A4FAA4188A1F861E861D868E01035F95
:1021A0001F4F9E01215F3F4F598B0E945C0D598943
:1021B00081119CC0D9824A825B83CC82BE82AD826F
:1021C00098868F82AE014F5F5F4F68E080E20E9489
:1021D000C60E2D853E85452D60E1C3010E94C70DC9
:1021E000182F81117FC0BD2CBB1CBB24BB1CE1146C
:1021F000F10409F46AC0EF85F8898281BB2009F4F3
:1022000055C0826082836401AA24A394C114D104BE
:1022100009F449C03C862B864D855E856F8578899B
:1022200087019E01255F3F4FC3010E94E00F182FD9
:102230008630B1F42F85388988EF298B3A8B0E943C
:102240002A0D85FB882780F98A2529893A89D901B1
:1022500012969C91129780FB91F912969C93D6CF7F
:10226000811140C0EBA5FCA53097A1F00190F08151
:10227000E02D0190F081E02DC4018C199D099A8711
:1022800089876B857C859E01275F3F4FA7018BA5C2
:102290009CA509958B859C85C81AD90A821593053A
:1022A00008F0B4CF12C011111DC014C08160828328
:1022B0004D855E8587019101BF01C3010E94F00E2B
:1022C000811114C02D853E850FC02D853E85B1102E
:1022D00003C00AC02D853E8560EA452DC3010E94DA
:1022E000C70D04C0812F02C060E8F7CF62960FB619
:1022F000F894DEBF0FBECDBFDF91CF911F910F913C
:10230000FF90EF90DF90CF90BF90AF909F908F9015
:102310007F906F905F904F903F902F9008958F9295
:102320009F92AF92BF92CF92EF920F931F931F9203
:102330001F921F930F933F932F934901A12CB12C10
:10234000CC24C394E12C06E020E80E94A7100F9053
:102350000F900F900F900F900F901F910F91EF9093
:10236000CF90BF90AF909F908F9008958F929F9243
:10237000AF92BF92CF92EF92FF920F931F921F9254
:10238000FF92EF923F932F934901A12CB12C22E0B1
:10239000C22EE02E06E020E80E94A7100F900F90BA
:1023A0000F900F900F900F900F91FF90EF90CF90A4
:1023B000BF90AF909F908F9008954F925F926F92D1
:1023C0007F928F929F92AF92BF92CF92DF92EF92C5
:1023D000FF920F931F93CF93DF93CDB7DEB7C05417
:1023E000D1090FB6F894DEBF0FBECDBF3C01D62E8B
:1023F000542E422EC02ECE0101965C017C01022F8C
:1024000029E030E0C3010E94B61181111BC08B800E
:102410009C801F93CF92BF92AF921F9280E48F93C4
:10242000A12CB12C82E0C82EE42C06E020E8452D3A
:102430006D2DC3010E94A7100F900F900F900F9069
:102440000F900F90C05CDF4F0FB6F894DEBF0FBE49
:10245000CDBFDF91CF911F910F91FF90EF90DF9053
:10246000CF90BF90AF909F908F907F906F905F9034
:102470004F9008958F929F92AF92BF92CF92EF921A
:102480000F93CF931F921F921F921F921F921F9222
:10249000812C912CA12CB12CC12CE22E05E020E046
:1024A0000E94A710C82F6CE271E080E090E00E94CB
:1024B000C90A0F900F900F900F900F900F908C2FD4
:1024C000CF910F91EF90CF90BF90AF909F908F9052
:1024D00008950F931F93CF93DF938A3F3FEF9307A6
:1024E00011F486ED2DC0DC011696ED91FC91179745
:1024F000EF2B09F1122F242FEC011A8740E00E94E4
:10250000870B082F8823C9F0682FCE010E94310C59
:10251000009739F3FC011483202F40E060E0CE01E6
:102520000E943A12182F882351F0602FCE010E948A
:10253000490C812F05C087ED03C084ED01C080E008
:10254000DF91CF911F910F9108952F923F924F925B
:102550005F926F927F928F929F92AF92BF92CF9233
:10256000DF92EF92FF920F931F93CF93DF93CDB73C
:10257000DEB766970FB6F894DEBF0FBECDBF1B8ADD
:1025800038E03C8B3CE33D8B8A3F3FEF930709F4F7
:10259000ADC0B22E342EA62E7C01DC011696CD9055
:1025A000DC901797CE01439617969C938E931697BF
:1025B0001A962C938E010F5F1F4F22E130E040E00E
:1025C00060E0C7010E948F11F701D782C682811196
:1025D000A5C069847A844B845C843D813E8B2E80C7
:1025E000670186E5C80ED11C460110E0D4018D912B
:1025F0009C91009789F1DC01ED91FC910084F185BB
:10260000E02D0995811128C0F40180819181DC01C0
:10261000ED91FC910088F189E02D622D09958823C8
:10262000D9F0F40180819181DC01ED91FC91048469
:10263000F585E02DA201B3010995811159C0F4017E
:1026400080819181DC01ED91FC910684F785E02D7C
:102650006E89099581114CC01F5FB2E08B0E911CF1
:10266000103121F610E0F60180819181009789F107
:10267000DC01ED91FC910084F185E02D099581113B
:1026800028C0F60180819181DC01ED91FC910088E8
:10269000F189E02D622D09958823A9F1F601808149
:1026A0009181DC01ED91FC910484F585E02DA2017E
:1026B000B301099581110DC0F60180819181DC0182
:1026C000ED91FC910684F785E02D6E8909958823AC
:1026D000D1F01F5FB2E0CB0ED11C103121F62B2DB3
:1026E000432D6A2DC7010E94691218C086ED16C0DD
:1026F0000B2D232D4A2D612FC7010E942A0E813DEB
:1027000009F4AACF0BC00B2D232D4A2D612FC70131
:102710000E942A0E982F977F913DD9F266960FB6A8
:10272000F894DEBF0FBECDBFDF91CF911F910F9107
:10273000FF90EF90DF90CF90BF90AF909F908F90E1
:102740007F906F905F904F903F902F9008958F9261
:102750009F92AF92BF92CF92EF920F931F921F92D0
:102760001F921F921F921F92812C912CA12CB12C91
:10277000C12CE22E09E020E00E94A7100F900F90DC
:102780000F900F900F900F900F91EF90CF90BF9000
:10279000AF909F908F900895AF92BF92CF92DF92AB
:1027A000EF92FF920F931F93CF93DF9300D000D04F
:1027B000CDB7DEB77C01690158011C821B821A82E9
:1027C00019828E010F5F1F4F9E012D5F3F4F0E94A8
:1027D0005C0D811109C049815A816B817C81850121
:1027E0009601C7010E94E00F0F900F900F900F907D
:1027F000DF91CF911F910F91FF90EF90DF90CF90DD
:10280000BF90AF900895AF92BF92CF92DF92EF92B8
:10281000FF920F931F93CF938C011D990EC088ECEC
:102820000E942A0D85FF05C0C8010E942F0860E2A2
:1028300001C060E088EC0E94420D8091A3018130CC
:1028400039F040F0823079F0833039F5C1E00CC0C6
:1028500083E106C08091F002807F8031F1F081E158
:102860008093F0021AC0C0E08091F002807F803136
:10287000A9F40E94C70ADC01CB0188539F4FAF4FD8
:10288000BF4F8093EC029093ED02A093EE02B093C1
:10289000EF0280E28093F00201C0C0E0780186E59B
:1028A000E80EF11C6801A6E7CA0ED11C5701F5011C
:1028B000819191915F01009739F0DC01ED91FC91DC
:1028C0000680F781E02D0995AC14BD0481F7909145
:1028D000F002903409F43FC050F4903221F190336B
:1028E000A1F1913109F084C0F60110820AC091353E
:1028F00009F458C0903809F46AC0903509F078C0DE
:1029000039C0D7018D919D917D01009739F0DC018F
:10291000ED91FC910480F581E02D0995EC14FD0406
:1029200081F782E163C00E94C70A0091EC02109116
:10293000ED022091EE023091EF02DC01CB01801B11
:10294000910BA20BB30BB7FD53C061E088EE0E9460
:10295000420D80E44BC088EE0E942A0D80FD48C0E5
:1029600088ED0E942A0D682F686088ED0E94420D54
:1029700080E53CC088EC0E942A0D86FF39C081E5C5
:102980008093F0020E94C70ADC01CB014496A11D8E
:10299000B11D8093EC029093ED02A093EE02B093F0
:1029A000EF0226C00E94C70AC090EC02D090ED0250
:1029B000E090EE02F090EF02DC01CB018C199D0952
:1029C000AE09BF09B7FD14C080E88093F0022C2F38
:1029D00040E060E0C8010E94A512882331F0823DEA
:1029E00039F08093F10280EA01C080E98093F0021F
:1029F000CF911F910F91FF90EF90DF90CF90BF90FC
:102A0000AF9008958F929F92AF92BF92CF92EF9224
:102A10000F93CF93DF93CDB7DEB7C054D1090FB674
:102A2000F894DEBF0FBECDBF5F934F939E012F5F23
:102A30003F4F3F932F931F9220E42F9320E8822E45
:102A4000912C5B0132E2C32EE12C06E021E840E04C
:102A5000FC016681848195810E94A7100F900F90E0
:102A60000F900F900F900F90C05CDF4F0FB6F8944F
:102A7000DEBF0FBECDBFDF91CF910F91EF90CF9012
:102A8000BF90AF909F908F9008958F929F92AF923A
:102A9000BF92CF92DF92EF92FF920F938E2CA42ED3
:102AA000B12C1F921F92DF92CF92FF92EF929F2C38
:102AB000C22EE02E09E021E2462FFC0166818481CE
:102AC00095810E94A7100F900F900F900F900F907C
:102AD0000F900F91FF90EF90DF90CF90BF90AF904D
:102AE0009F908F9008958F929F92AF92BF92CF92B6
:102AF000EF920F93A62EB12C1F921F921F921F923E
:102B00001F921F92812C912CC22EE42E0AE021E20A
:102B100040E0FC016681848195810E94A7100F909E
:102B20000F900F900F900F900F900F91EF90CF900C
:102B3000BF90AF909F908F9008958F929F92AF9289
:102B4000BF92CF92EF920F93A62EB12C1F921F929D
:102B50001F921F921F921F92812C912CC12CE42E48
:102B60000BE021E240E0FC016681848195810E94B6
:102B7000A7100F900F900F900F900F900F900F9144
:102B8000EF90CF90BF90AF909F908F900895FC01F1
:102B90008285089581E0693009F080E00895CF933F
:102BA000DF93EC018A819B81DC01ED91FC91048033
:102BB000F581E02D6A8509958A85813439F4EA81A9
:102BC000FB81EA58FF4F8081846080831A861B86D0
:102BD0001C861D861E861F86188A80E0DF91CF9195
:102BE00008958F929F92AF92BF92CF92EF920F93E0
:102BF000A42EB12CB22A1F921F921F921F921F92D5
:102C00001F92812C912CC12CE62E01E023E240E0A2
:102C1000FC016285828193810E94A7100F900F9022
:102C20000F900F900F900F900F91EF90CF90BF905B
:102C3000AF909F908F9008958F929F92AF92BF9286
:102C4000CF92EF920F93A62EB12C1F921F923F931B
:102C50002F935F934F934A01C12CE12C00E023EAAC
:102C600040E0FC016285828193810E94A7100F9051
:102C70000F900F900F900F900F900F91EF90CF90BB
:102C8000BF90AF909F908F9008958F929F92AF9238
:102C9000BF92CF92EF920F93A42EB12CB22A1F9223
:102CA0001F921F921F921F921F92812C912CC12C58
:102CB000E62E03E023E240E0FC01628582819381FD
:102CC0000E94A7100F900F900F900F900F900F90F1
:102CD0000F91EF90CF90BF90AF909F908F900895FD
:102CE0002F923F924F925F926F927F928F929F921C
:102CF000AF92BF92CF92DF92EF92FF920F931F930A
:102D0000CF93DF93CDB7DEB7E8970FB6F894DEBF69
:102D10000FBECDBFDC011296ED90FC9013971A9672
:102D20003C91311104C1122F242E362E3C01D701C3
:102D3000ED91FC910190F081E02D60E0C7010995D3
:102D40006C01009709F4F5C0FC01A080B180A114CA
:102D5000B10409F4F0C04301F4E08F0E911CDC01D2
:102D600011969C928E9214961C93FE0131962F011F
:102D70008F0128E030E040E060E0D30112968D91B1
:102D80009C9113970E948F11F60114828111D9C072
:102D900009818D81893009F0D0C0D701ED91FC9176
:102DA0000280F381E02D222D41E0632DC7010995BA
:102DB000F3018287882309F4C2C098859583282F60
:102DC00040E060E0828193810E943A12182F8823AC
:102DD00089F0D601AD92BC92D701ED91FC910480AF
:102DE000F581E02DD3011A966C91C7010995F30185
:102DF0001286ABC0202F013208F020E2D601AD923E
:102E0000BC9221110BC0940142E0F30162858281E2
:102E100093810E94C90C811197C010C030E08201DB
:102E200040E0D3011A966C911A9712968D919C915D
:102E300013970E948F11811187C0E5CF1F921F92B7
:102E40005F924F921F9288E08F9388E0882E912C9A
:102E5000A12CB12C99E2C92EE12C06E020EA40E039
:102E6000F3016285828193810E94A710182F0F9031
:102E70000F900F900F900F900F90811166C08B8173
:102E8000D3011B968C931B97720100E028E030E081
:102E900040E01A966C911A9712968D919C91139717
:102EA0000E94B611811150C02B813C8140E0F3019A
:102EB0006285828193810E94B611811145C029816A
:102EC00030E0CE0181967C0140E0D3011A966C91EE
:102ED0001A9712968D919C9113970E94B6118111A9
:102EE00033C02E8140E0F3016285828193810E948C
:102EF000A713811129C001E0D3011B968C911B9768
:102F0000801740F020E0402F68E0C3010E94451682
:102F10000F5FF2CF1296ED91FC911397EA58FF4F95
:102F200080818460808381E050968C930EC019ED7F
:102F30000CC016ED0AC017ED08C011ED06C014ED67
:102F400004C0F601B182A082182F812FE8960FB637
:102F5000F894DEBF0FBECDBFDF91CF911F910F91CF
:102F6000FF90EF90DF90CF90BF90AF909F908F90A9
:102F70007F906F905F904F903F902F900895CF92E9
:102F8000DF92FF920F931F93CF93DF9300D000D077
:102F9000CDB7DEB78C01F62E19821A821B821C82F5
:102FA00020E0462F61E10E94F11520E04F2D60E105
:102FB000C8010E94F11520E04F2D64E0C8010E9475
:102FC000451683E0C82ED12C9E012F5F3F4F44E071
:102FD00050E06F2DC8010E941C168823F1F020E0FC
:102FE0004F2D64E1C8010E94F11520E04F2D60E1F2
:102FF000C8010E94F11564E170E080E090E00E9459
:10300000C90A0F900F900F900F90DF91CF911F91F1
:103010000F91FF90DF90CF90089589819A81AB81C5
:10302000BC819D7F83309140A041B105C1F264E62F
:1030300070E080E090E00E94C90A81E0C81AD108DF
:1030400019F6CDCFFC0182E791E0918380837383F1
:103050006283128613861486158616861786108A52
:10306000148288E085839CE3968391E09783808730
:1030700084E0818761157105B1F0DB01AA5ABF4F69
:1030800080E090E02D913D91232B49F48B96880FA1
:10309000991FDB01A80FB91FED93FC9308950196CA
:1030A0008031910579F70895EF92FF920F931F9366
:1030B000CF938C01C62F7A01FA0180819181A28180
:1030C000B3818130F3E09F07F1E0AF07B105D1F0A4
:1030D00060F48115E1E09E07AE07B10571F1813022
:1030E0009140A140B10571F064C0833021E09207A6
:1030F00020E1A207B105E1F183309340A041B10581
:10310000B9F157C08091F202811153C020E04C2FD9
:1031100061E1C8010E94F11520E04C2F60E1C80177
:103120000E94F11520E04C2F64E0C8010E94451672
:1031300081E08093F20281EB3DC020E0462F61E107
:10314000C8010E94F11520E04C2F60E1C8010E94E7
:10315000F1151092F202F80162856770C770660F70
:10316000660F660F6C2B828193810E94E60C21C052
:1031700020E04C2F64E1C8010E94F11520E04C2FA3
:1031800060E1C8010E94F11564E170E080E090E028
:103190000E94C90AF8016285F701218126952170F4
:1031A00067704C2FF801828193810E94A5121092C2
:1031B000F20280E0CF911F910F91FF90EF90089560
:1031C000EF92FF920F931F93CF93DF93CDB7DEB7AC
:1031D0002E970FB6F894DEBF0FBECDBF7C0181E005
:1031E00090E09E878D878E010F5F1F4F9E01235FAA
:1031F0003F4F41E0F7016285828193810E94CC13A9
:10320000811151C002E011E089818023D1F019863B
:103210001A861B861C869E01275F3F4F44E050E0C4
:10322000612FC7010E941C1681110BC0AE01475FC0
:103230005F4F612FC7010E945418813B99F18111A2
:1032400032C0000F1F5F1830F9F611E0F7018385D7
:10325000811740F119861A861B861C869E01275FFE
:103260003F4F44E050E0612FC7010E941C168111BE
:1032700017C089859A85877091708130914081F45B
:103280008B859C8581609C878B87AE01475F5F4FF4
:10329000612FC7010E945418813B21F0811103C0A6
:1032A0001F5FD4CF80E02E960FB6F894DEBF0FBE1E
:1032B000CDBFDF91CF911F910F91FF90EF900895B7
:1032C0000F931F93CF93DF93FC012089211102C03C
:1032D00080E020C0EC010E94C70A0C851D852E8568
:1032E0003F85DC01CB01801B910BA20BB30BB7FD1B
:1032F000EFCFCE010E94E018182F0E94C70ADC0110
:10330000CB018C599F4FAF4FBF4F8C879D87AE87A6
:10331000BF87812FDF91CF911F910F910895CF9398
:10332000DF93FC01EA0180819181892B19F580E00E
:1033300027C028813981232BD1F3DB012D913C91CA
:10334000D9019C91A381B0E0A81BB10920813181F2
:10335000A20FB31F9C9382818150828388819981BF
:10336000019799838883DB018D919C911197019638
:103370008D939C9382818111DCCF8381828381E054
:10338000DF91CF910895CF92DF92EF92FF920F934A
:103390001F93CF93DF936C01EB017B01E40EF51ECD
:1033A00000E010E0CE15DF0561F06991D601ED91E6
:1033B000FC910190F081E02DC6010995080F191FBD
:1033C000F1CFC801DF91CF911F910F91FF90EF9046
:1033D000DF90CF9008958091FF0208959FB7F894F1
:1033E0001092F6029FBF90918204943009F057C06A
:1033F0009091E9009F703091EC00232F217030FDF7
:1034000020E8922B24E02093E9002091EB0020FF9C
:1034100043C02091EE0027FF3FC02091F3022223FA
:1034200021F02091E80025FF37C01092F30226E03A
:103430003091E80035FD15C030918204343061F5DB
:103440003091EB0035FD28C0215021F481E08093BC
:10345000F30222C0EFE9FFE03197F1F700C000006E
:10346000E7CF8093F1008091E80085FD0AC080914C
:10347000E80080FFFCCF8091E8008E778093E80021
:1034800006C08FB7F89421E02093F6028FBF9F709B
:103490009093E90080E008959F709093E9008FEF8A
:1034A0000895CF93DF9300D01F92CDB7DEB79C0174
:1034B00080918204843019F593E099833B832A83B9
:1034C0009093E9008FEF9091E800815095FD06C040
:1034D00095ED9A95F1F700008111F5CF8091E80004
:1034E00085FF0DC040E050E063E070E0CE01019642
:1034F0000E949B1C8091E8008E778093E8000F90DB
:103500000F900F90DF91CF910895CF93DF9300D06C
:103510001F92CDB7DEB720918204243021F522E03E
:1035200029839B838A8383E08093E9008FEF9091C6
:10353000E800815095FD06C095ED9A95F1F70000E1
:103540008111F5CF8091E80085FF0DC040E050E08B
:1035500063E070E0CE0101960E949B1C8091E80020
:103560008E778093E8000F900F900F90DF91CF91AE
:103570000895209182042430F1F422E02093E900A0
:103580002FEF3091E800215035FD06C035ED3A951A
:10359000F1F700002111F5CF2091E80025FF0BC0C5
:1035A00040E050E065E070E00E949B1C8091E800E4
:1035B0008E778093E8000895CF93DF932091820463
:1035C000243039F521E02093E9002FEF3091E80015
:1035D000215035FD06C035ED3A95F1F70000211177
:1035E000F5CF2091E80025FF14C0EC0140E050E049
:1035F00068E070E00E949B1C8091E8008E778093C9
:10360000E80088E0FE01A7EFB2E001900D928A95F4
:10361000E1F7DF91CF9108958EE692E00E94BD021E
:1036200080918104811109C00E94301E0E948D1E6C
:103630008091E20084608093E20008958AE692E03F
:103640000E94BD0210928104089508952091F40211
:103650002F5F822F62E30E94AE31992319F02093ED
:10366000F40208951092F4028091F602882371F119
:1036700080918204843041F58091E9008F7020911F
:10368000EC00922F917020FD90E8892B94E09093AC
:10369000E9009091EB0090FF14C09091EE0097FF2D
:1036A00010C09091E80095FF03C01092F100F9CF8F
:1036B0009091E80090FF05C09091E8009E7790936C
:1036C000E8008F708093E9001092F602089542E0BE
:1036D00061EC81E00E94AA1D42E061EC82E00E9460
:1036E000AA1D42E061EC83E00E94AA1D42E261EC67
:1036F00084E00C94AA1D80918404833009F453C0A3
:1037000030F4813071F0823009F48CC008958A3031
:1037100009F478C08B3009F45EC0893009F09AC092
:1037200020C080918304813A09F094C08091E80020
:10373000877F8093E8008091870490918804892B8B
:1037400021F468E087EF92E003C060E080E090E061
:1037500070E00E94E61C8091E8008B778093E8007F
:10376000089580918304813209F074C080918704A8
:1037700090918804892B09F06DC08091E800877FC3
:103780008093E8008091E80082FD05C0809182046A
:103790008111F8CF5FC08091F1008093FF0280918A
:1037A000E8008B7753C080918304813A09F052C0BE
:1037B0008091870490918804892B09F04BC08091F7
:1037C000E800877F8093E8008091E80080FFFCCFCD
:1037D00080910A0136C0809183048132D9F58091AD
:1037E000870490918804892BA9F58091E800877F50
:1037F0008093E8000E94DF1D8091850480930A0178
:103800000C94C72680918304813221F58091E800D1
:10381000877F8093E8000E94DF1D8091860480935B
:103820000003089580918304813AA1F48091E80017
:10383000877F8093E8008091E80080FFFCCF809133
:1038400000038093F1008091E8008E778093E80078
:103850000C94DF1D08958091FF028093F502109271
:10386000FF0280E00E94A4070E94A4220C94C726B5
:103870000C942B1C0E94392D8091F5028093FF023D
:1038800008950C943A1C292F332723303105C9F0B1
:1038900064F42130310581F02230310509F043C054
:1038A00084E790E024EC32E042C021323105F1F0AF
:1038B0002232310541F137C082E190E028E333E064
:1038C00036C099278130910541F08230910541F051
:1038D000892B49F5E0ECF2E005C0E0EBF2E002C034
:1038E000E2E7F2E0849190E09F0121C06430D8F4D7
:1038F000E62FF0E0EE0FFF1FE057FE4F20813181F1
:1039000089E090E014C0643070F470E0FB01EE0FC9
:10391000FF1FE857FE4F20813181FB01EC57FE4F1E
:10392000808190E004C080E090E020E030E0FA0187
:10393000318320830895CF92DF92EF92FF920F930D
:103940001F93CF93DF93EC018B016A010E94FE1D50
:10395000811133C0C114D10439F0F6018081918105
:10396000081B190BC80FD91FE12CF12C01151105EB
:1039700019F18091E80085FD16C08091E8008E77EE
:103980008093E800C114D10449F0F601808191814F
:10399000E80EF91EF182E08285E00FC00E94FE1D54
:1039A000882321F30AC089918093F1000150110905
:1039B000FFEFEF1AFF0ADACF80E0DF91CF911F917E
:1039C0000F91FF90EF90DF90CF90089520918904A0
:1039D00030918A042617370748F06115710539F4CC
:1039E0002091E8002E772093E80001C0B90140E063
:1039F00061157105A9F120918204222309F443C0C5
:103A0000253009F442C02091E80023FD40C02091F8
:103A1000E80022FD32C02091E80020FFE9CF40916C
:103A2000F3002091F20030E0342BFC01CF0161154E
:103A3000710559F02830310540F481918093F100EF
:103A4000615071092F5F3F4FF1CF41E028303105C0
:103A500009F040E02091E8002E772093E800C8CFDD
:103A60004111C9CF0AC080918204882361F085305A
:103A700061F08091E80083FD0AC08091E80082FF38
:103A8000F2CF80E0089582E0089583E0089581E018
:103A900008952091890430918A042617370748F049
:103AA0006115710539F42091E8002E772093E80024
:103AB00001C0B901FC0120E06115710591F180910F
:103AC0008204882309F440C0853009F43FC0809106
:103AD000E80083FD3DC08091E80082FD2FC0809109
:103AE000E80080FFE9CF2091F3008091F20090E0A0
:103AF000922B6115710559F08830910540F424919D
:103B00002093F1003196615071090196F2CF21E0C6
:103B1000089709F020E08091E8008E778093E80014
:103B2000CBCF2111CCCF0AC080918204882361F0D1
:103B3000853061F08091E80083FD0AC08091E80043
:103B400082FFF2CF80E0089582E0089583E0089537
:103B500081E00895982F973058F59093E9009817D1
:103B600039F07091EC002091ED005091F00003C00D
:103B7000242F762F50E021FF19C03091EB003E7FBB
:103B80003093EB003091ED003D7F3093ED003091AC
:103B9000EB0031603093EB007093EC002093ED006C
:103BA0005093F0002091EE0027FF07C09F5FD3CF16
:103BB0008F708093E90081E0089580E008958091FE
:103BC000830487FF11C08091E80082FD05C08091C9
:103BD00082048111F8CF11C08091E8008B770BC06F
:103BE00080918204882349F08091E80080FFF8CF1B
:103BF0008091E8008E778093E80008952091E4009A
:103C00003091E50095E64091EC00842F817040FFF3
:103C100022C08091E80080FD1CC08091820488232E
:103C200091F0853091F08091EB0085FD10C04091BE
:103C3000E4005091E5004217530729F39A0191508F
:103C400011F784E0089582E0089583E0089581E00B
:103C5000089580E008954091E80042FFDECF089586
:103C60000E949E1E0E94A61EE0EEF0E08081816010
:103C70008083E8EDF0E080818F77808319BCA7ED29
:103C8000B0E08C918E7F8C9380818F7E80831092A8
:103C9000810408950F931F93CF93DF930E949E1E7C
:103CA0000E94A61EC8EDD0E088818F778883888126
:103CB0008068888388818F7D888319BC10928204F4
:103CC00010927E041092800410927F0400EE10E0A7
:103CD000F80180818B7F808388818160888342E0C6
:103CE00060E080E00E94AA1DE1EEF0E080818E7F1E
:103CF0008083E2EEF0E08081816080838081886053
:103D00008083F80180818E7F8083888180618883B1
:103D1000DF91CF911F910F910895E8EDF0E0808140
:103D20008F7E8083E7EDF0E080818160808384E096
:103D300082BF81E0809381040C944A1EE8EDF0E09C
:103D400080818E7F80831092E20008951092DA00C5
:103D50001092E10008951F920F920FB60F92112456
:103D60002F933F934F935F936F937F938F939F9383
:103D7000AF93BF93EF93FF938091E10082FF0BC05D
:103D80008091E20082FF07C08091E1008B7F8093E9
:103D9000E1000E94261B8091DA0080FF1FC0809105
:103DA000D80080FF1BC08091DA008E7F8093DA00FC
:103DB0008091D90080FF0DC080E189BD82E189BD7D
:103DC00009B400FEFDCF81E0809382040E940C1BA9
:103DD00005C019BC109282040E941E1B8091E10054
:103DE00080FF19C08091E20080FF15C08091E20041
:103DF0008E7F8093E2008091E20080618093E200F8
:103E00008091D80080628093D80019BC85E08093AF
:103E100082040E94381C8091E10084FF30C08091B0
:103E2000E20084FF2CC080E189BD82E189BD09B434
:103E300000FEFDCF8091D8008F7D8093D8008091C7
:103E4000E1008F7E8093E1008091E2008F7E80937D
:103E5000E2008091E20081608093E20080917E0424
:103E6000882311F084E007C08091E30087FD02C041
:103E700081E001C083E0809382040E94411C809114
:103E8000E10083FF29C08091E20083FF25C080917B
:103E9000E100877F8093E10082E0809382041092AA
:103EA0007E048091E1008E7F8093E1008091E200AA
:103EB0008E7F8093E2008091E20080618093E20037
:103EC00042E060E080E00E94AA1D8091F0008860DE
:103ED0008093F0000E94251BFF91EF91BF91AF915D
:103EE0009F918F917F916F915F914F913F912F9112
:103EF0000F900FBE0F901F9018951F920F920FB644
:103F00000F9211242F933F934F935F936F937F935F
:103F10008F939F93AF93BF93CF93DF93EF93FF93D1
:103F2000C091E900CF708091EC00D82FD17080FD56
:103F3000D0E81092E9008091F000877F8093F00034
:103F400078940E94C11F1092E9008091F00088606F
:103F50008093F000CD2BCF70C093E900FF91EF91DB
:103F6000DF91CF91BF91AF919F918F917F916F9191
:103F70005F914F913F912F910F900FBE0F901F9027
:103F800018951F93CF93DF93CDB7DEB7AA970FB6DF
:103F9000F894DEBF0FBECDBFE3E8F4E088E08E0FFB
:103FA0009091F10091938E13FBCF0E947B1B809127
:103FB000E80083FF1FC18091830490918404492FFE
:103FC00050E04A30510508F015C1FA01EA5AFF4F96
:103FD0000C94CE31803881F0823809F00BC1809189
:103FE00087048F708093E9008091EB0085FB882720
:103FF00080F91092E90006C080917F0490918004BE
:10400000911182609091E800977F9093E8008093EF
:10401000F1001092F100C8C0282F2D7F09F0EAC0EE
:10402000882319F0823061F0E5C0809185048130E9
:1040300009F0E0C0933009F080E0809380042BC049
:1040400080918504811127C0809187048F7009F4C5
:10405000D1C08093E9002091EB0020FF1CC0933079
:1040600021F48091EB00806214C09091EB0090618C
:104070009093EB0021E030E0A90102C0440F551FEE
:104080008A95E2F74093EA001092EA008091EB00F3
:1040900088608093EB001092E9008091E800877FB0
:1040A00086C08111A7C0109185041F778091E3001D
:1040B0008078812B8093E3008091E800877F809354
:1040C000E8000E94DF1D8091E80080FFFCCF809116
:1040D000E30080688093E300111102C082E001C018
:1040E00083E08093820486C08058823008F082C0CA
:1040F00080918504909186048C3D53E0950779F575
:1041000083E08A838AE289834FB7F894DE011396AD
:1041100020E03EE051E2E32FF0E050935700E491BD
:1041200020FF03C0E295EF703F5FEF708E2F90E0AD
:10413000EA3010F0C79601C0C0968D939D932F5F13
:10414000243149F74FBF8091E800877F8093E800D2
:104150006AE270E0CE0101960E94E61C14C0AE0136
:104160004F5F5F4F609187040E94431CBC01892B05
:1041700009F440C09091E800977F9093E80089810E
:104180009A810E94491D8091E8008B778093E80016
:1041900031C0803879F58091E800877F8093E8000E
:1041A00080917E048093F1008091E8008E77809367
:1041B000E8000E94DF1D1EC081111CC09091850483
:1041C0009230C0F48091E800877F8093E80090935C
:1041D0007E040E94DF1D80917E04811106C08091C3
:1041E000E30087FD02C081E001C084E08093820487
:1041F0000E94671B8091E80083FF0AC08091E8005D
:10420000877F8093E8008091EB0080628093EB00D1
:10421000AA960FB6F894DEBF0FBECDBFDF91CF9147
:104220001F91089590930603809305030895E091EC
:104230000503F0910603309721F00190F081E02D05
:10424000099480E00895EF92FF920F931F93CF930C
:10425000DF93E0910503F09106033097B1F18C01F3
:104260000280F381E02D09958091730482FF2DC0B7
:1042700080FF04C085E594E00E94BD02E80118E0DB
:104280008FE4E82E84E0F82E8091730480FF0BC049
:1042900088811F928F93FF92EF920E9456030F9096
:1042A0000F900F900F90115021961111EDCF80912A
:1042B000730480FF0AC08DE494E0DF91CF911F91D9
:1042C0000F91FF90EF900C94BD02DF91CF911F9161
:1042D0000F91FF90EF900895E0910503F091060390
:1042E000309721F00480F581E02D09940895CF9353
:1042F000DF93EC018091030390910403C817D90761
:1043000009F1D0930403C0930303E0910503F091F6
:1043100006033097B9F00680F781E02DCE010995AC
:104320008091730482FF0EC080FF0CC0DF93CF9397
:104330008FE394E09F938F930E9456030F900F900A
:104340000F900F90DF91CF910895CF93DF93EC0101
:104350008091010390910203C817D90709F1D09306
:104360000203C0930103E0910503F0910603309727
:10437000B9F00084F185E02DCE0109958091730498
:1043800082FF0EC080FF0CC0DF93CF938FE294E0DA
:104390009F938F930E9456030F900F900F900F9052
:1043A000DF91CF9108950E94170B0C94AB085F9298
:1043B0006F927F928F929F92AF92BF92CF92DF9235
:1043C000EF92FF920F931F93CF93DF9300D000D013
:1043D0001F92CDB7DEB70E94080608E013E0512C0B
:1043E00088248394912C852D0E943A075C01F80162
:1043F000C080D180C826D926C114D10439F4539481
:104400000E5F1F4FF0E15F12EECF3FC0809173044B
:1044100081FD0E946A07E12CF12C34010E2C02C0B0
:10442000660C771C0A94E2F7C3018C219D21892B2D
:1044300021F1E9825A8221E0C3018A219B21892B43
:1044400009F420E02B830E94200B8160782F9D834C
:104450008C8349815A816B818D810E94A52249817B
:104460005A816B817C818D810E94262DF80180818B
:1044700091816826792671826082FFEFEF1AFF0A28
:1044800080E1E816F10449F6BACF8FEF89838A8379
:104490001B820E94200B8160782F9D838C83498131
:1044A0005A816B818D810E94A5220E94252D0E9438
:1044B0009E2F109107030E941721181771F10E9477
:1044C0001721809307039091730492FF0EC090FF11
:1044D0000CC01F928F9380E694E09F938F930E946D
:1044E00056030F900F900F900F90809107030F903D
:1044F0000F900F900F900F90DF91CF911F910F9120
:10450000FF90EF90DF90CF90BF90AF909F908F90F3
:104510007F906F905F900C94372D0F900F900F90BD
:104520000F900F90DF91CF911F910F91FF90EF901F
:10453000DF90CF90BF90AF909F908F907F906F90C3
:104540005F9008950C94A4070895CF93DF93CDB79F
:10455000DEB72B970FB6F894DEBF0FBECDBF942FFA
:104560004F83252F588769877A878B874A855B8594
:10457000452B21F02F3F09F59F3FF9F4DE011196FD
:1045800086E0FD0111928A95E9F785E0FE013796F4
:1045900001900D928A95E1F749815A816B817C8166
:1045A0008D819E810E9492292B960FB6F894DEBFD2
:1045B0000FBECDBFDF91CF9108954F81588569859A
:1045C0007A858B850E94262DD9CF882309F45CC07B
:1045D0009CEF980F913A20F090E5980F9E3218F4D6
:1045E0000E94512C0DC090E2980F983058F48770BB
:1045F00091E001C0990F8A95EAF7892F0E94902CCB
:104600000C94CA2C9BE5980F933070F4853A29F0EE
:10461000863A31F083E890E005C081E890E002C07E
:1046200082E890E00C94772198E5980F953160F539
:10463000883A89F0893A91F08A3A99F08B3AA1F058
:104640008C3AA9F08D3AB1F08E3AB9F08F3AC1F0B8
:1046500080E090E017C082EE90E014C089EE90E018
:1046600011C08AEE90E00EC085EB90E00BC086EBA7
:1046700090E008C083EB90E005C084EB90E002C0BE
:1046800087EB90E00C94A5210895882349F19CEFD5
:10469000980F913A20F090E5980F9E3218F40E94FE
:1046A0006E2C0DC090E2980F983058F4877091E00E
:1046B00001C0990F8A95EAF7892F0E94962C0C94D5
:1046C000CA2C9BE5980F933020F480E090E00C9486
:1046D0007721885A853120F480E090E00C94A52160
:1046E0000895882321F00E94902C0C94CA2C0895E0
:1046F000882321F00E94962C0C94CA2C0895BF9216
:10470000CF92DF92EF92FF920F931F93CF93DF939D
:1047100000D000D000D0CDB7DEB725E0FC01DE012F
:10472000119601900D922A95E1F7FC01408151818B
:10473000028163817481258122952F706115710535
:1047400009F403C35F3F19F44F3F09F4FEC26C0143
:10475000862F7D836C83602F782F8D812E830E941E
:10476000E42B182FB92E0E94E32B0E94DD2AEB2D9B
:10477000E295EF70F0E0E05AFF4F2E810C94CE31BD
:104780008B2D807F9B2D9F70F92E882319F0F2943A
:1047900090EFF922002349F0FF2009F483C28F2D06
:1047A0000E94A32C0E94CA2C7DC2812F0E94452307
:1047B000FF2009F4CAC28F2D0E94A92C26960FB69D
:1047C000F894DEBF0FBECDBFDF91CF911F910F9147
:1047D000FF90EF90DF90CF90BF900C94CA2C8B2D60
:1047E000807F9B2D9F70F92E803219F0F29480EF1C
:1047F000F822112319F0113009F12AC00023B1F079
:104800008F2D222351F1213041F526960FB6F894D1
:10481000DEBF0FBECDBFDF91CF911F910F91FF90F3
:10482000EF90DF90CF90BF900C94B32C222319F01F
:10483000213009F48AC20E94B62C2DC00023F1F069
:10484000263008F082C20E948D2C8F2129F023C0CF
:104850000023F9F0211116C08F2D26960FB6F8947B
:10486000DEBF0FBECDBFDF91CF911F910F91FF90A3
:10487000EF90DF90CF90BF900C947123253008F01B
:1048800064C209C0F601858180FF0CC28F708583E8
:10489000E3CF21111CC28F2D83C12B2D2695269588
:1048A000237030E02115310521F021303105D1F0A0
:1048B0004CC2002321F0812F9B2D937002C080E019
:1048C00090E026960FB6F894DEBF0FBECDBFDF9105
:1048D000CF911F910F91FF90EF90DF90CF90BF90FD
:1048E0000C947721002321F0812F9B2D937002C01F
:1048F00080E090E026960FB6F894DEBF0FBECDBFE5
:10490000DF91CF911F910F91FF90EF90DF90CF90AB
:10491000BF900C94A521812F002319F00E94242E12
:1049200002C00E948C2E26960FB6F894DEBF0FBEF2
:10493000CDBFDF91CF911F910F91FF90EF90DF904E
:10494000CF90BF900C94112F8B2D837009F07BC0FA
:104950000111FBC1812F829586958770880F880F82
:10496000912F9F70C92ED12CE12CF12C082E04C060
:10497000CC0CDD1CEE1CFF1C0A94D2F714FF12C0F5
:104980004FE050E060E070E004C0440F551F661F28
:10499000771F8A95D2F7CB01BA0160957095809503
:1049A000909503C060E070E0CB012B2D26952695F5
:1049B0002370422F50E042305105D9F04330510569
:1049C00069F16C297D298E299F294130510551F1CA
:1049D00026960FB6F894DEBF0FBECDBFDF91CF9104
:1049E0001F910F91FF90EF90DF90CF90BF900C94AC
:1049F000F82A6C297D298E299F2926960FB6F894CE
:104A0000DEBF0FBECDBFDF91CF911F910F91FF9001
:104A1000EF90DF90CF90BF900C94122B0E94F82A59
:104A2000C701B60126960FB6F894DEBF0FBECDBF04
:104A3000DF91CF911F910F91FF90EF90DF90CF907A
:104A4000BF900C94DE2A002319F08B2D817001C0D9
:104A50008695882309F479C1812F82958695877080
:104A6000880F880F912F9F70C92ED12CE12CF12C2B
:104A7000082E04C0CC0CDD1CEE1CFF1C0A94D2F7DF
:104A800014FF12C04FE050E060E070E004C0440F3B
:104A9000551F661F771F8A95D2F7CB01BA01609523
:104AA00070958095909503C060E070E0CB012B2D50
:104AB000269526952370422F50E042305105D9F0BB
:104AC0004330510569F16C297D298E299F29413098
:104AD000510551F126960FB6F894DEBF0FBECDBF3B
:104AE000DF91CF911F910F91FF90EF90DF90CF90CA
:104AF000BF900C94BF2B6C297D298E299F29269667
:104B00000FB6F894DEBF0FBECDBFDF91CF911F91DE
:104B10000F91FF90EF90DF90CF90BF900C94D12B2E
:104B20000E94BF2BC701B60126960FB6F894DEBFD0
:104B30000FBECDBFDF91CF911F910F91FF90EF90EE
:104B4000DF90CF90BF900C94AD2B103FD1F128F4A3
:104B500080E4810F803250F0A0C0123F09F462C09F
:104B600008F44BC0133F09F472C097C0F12FF071E5
:104B7000FF2E8B2D8F71002351F00E94462B812F29
:104B8000FF2019F08295807F68CE8F7066CE0E94DC
:104B9000672B812FFF2019F08295807F01C08F70D5
:104BA00026960FB6F894DEBF0FBECDBFDF91CF9132
:104BB0001F910F91FF90EF90DF90CF90BF900C94DA
:104BC00078230023B1F0253008F0BFC08B2D8F7102
:104BD00026960FB6F894DEBF0FBECDBFDF91CF9102
:104BE0001F910F91FF90EF90DF90CF90BF900C94AA
:104BF0008C2B263008F0A9C0E9CF0023A9F08B2D1B
:104C00008F7126960FB6F894DEBF0FBECDBFDF9131
:104C1000CF911F910F91FF90EF90DF90CF90BF90B9
:104C20000C94462B002359F38B2D8F7126960FB6CB
:104C3000F894DEBF0FBECDBFDF91CF911F910F91D2
:104C4000FF90EF90DF90CF90BF900C94672B0023E4
:104C500099F08B2D8F7126960FB6F894DEBF0FBE9C
:104C6000CDBFDF91CF911F910F91FF90EF90DF901B
:104C7000CF90BF900C94312B26960FB6F894DEBFE0
:104C80000FBECDBFDF91CF911F910F91FF90EF909D
:104C9000DF90CF90BF900C942C2B0023A9F02223FF
:104CA00009F4ADCF812F26960FB6F894DEBF0FBE64
:104CB000CDBFDF91CF911F910F91FF90EF90DF90CB
:104CC000CF90BF900C94E522222309F4ADCF812F21
:104CD00026960FB6F894DEBF0FBECDBFDF91CF9101
:104CE0001F910F91FF90EF90DF90CF90BF900C94A9
:104CF00045234B2D4F70612FC6010E949E2D269695
:104D00000FB6F894DEBF0FBECDBFDF91CF911F91DC
:104D10000F91FF90EF90DF90CF90BF900C94362AC8
:104D20004B2D4F70612FC60126960FB6F894DEBF4B
:104D30000FBECDBFDF91CF911F910F91FF90EF90EC
:104D4000DF90CF90BF900C94A12D26960FB6F894CB
:104D5000DEBF0FBECDBFDF91CF911F910F91FF90AE
:104D6000EF90DF90CF90BF9008950E94B02C0E94EA
:104D70007F2C0E94CA2C0E9443300E94112F80E099
:104D800090E00E94772180E090E00C94A5210E94A1
:104D9000A02C0C94B526CF93DF9300D000D01F92A7
:104DA000CDB7DEB70E94E42B292F22952F7030E07B
:104DB0002C3031054CF42A303105C4F4225031092D
:104DC0002230310540F023C02C303105D1F02F3096
:104DD0003105B9F01CC0853A28F48430B0F4823033
:104DE00028F413C090E2980F983078F0883E30F4A1
:104DF000803E58F48450813A50F407C0803F39F423
:104E000004C093FB882780F903C081E001C080E0E3
:104E10000F900F900F900F900F90DF91CF9108950A
:104E2000CF93DF9300D000D01F92CDB7DEB70F90A5
:104E30000F900F900F900F90DF91CF910895CF9327
:104E4000DF9300D000D000D0CDB7DEB726960FB6E6
:104E5000F894DEBF0FBECDBFDF91CF9108951F93B1
:104E6000CF93DF93C091280316E080912903C817E0
:104E700099F0D0E01C9FF0011D9FF00D1124E65D1C
:104E8000FC4F4081518162817381848195810E94B0
:104E90001F272196C770E9CFDF91CF911F91089509
:104EA00040915A0350915B0360915C0370915D03E4
:104EB00080915E0390915F030C941F2780915F03A4
:104EC00082958F7009F054C080915C03882309F4A7
:104ED0004FC080912803A091290360915A037091DB
:104EE0005B0340915D0350915E03B6E08A1709F4BD
:104EF0003FC090E041155105C1F17F3F11F46F3F74
:104F0000A1F1B89FF001B99FF00D1124E65DFC4FAF
:104F1000218172132AC02081621327C022812111AE
:104F200024C0238134812417350710F4215031091E
:104F3000241B350B283C3105C0F420915F032F70F2
:104F4000206120935F0326E0289FF001299FF00D48
:104F50001124E15DFC4F80818F70806180838AE540
:104F600093E00E947F230C942F2701968770BECF79
:104F70000895BF92CF92DF92EF92FF920F931F930B
:104F8000CF93DF93CDB7DEB761970FB6F894DEBF4E
:104F90000FBECDBF7C0185E0F701DE011D960190BB
:104FA0000D928A95E1F7D7014C9111965C9111977A
:104FB0001296DC90129713960D911C9114973091D4
:104FC0005A0360915B0380915D0390915E030097AB
:104FD00009F477C16F3F19F43F3F09F472C1B090F3
:104FE0005C03BB2009F4C5C020915F0308171907B3
:104FF00028F0F801E81BF90BCF0104C080959095CB
:10500000800F911FCC24C394883C910580F0C12C63
:10501000207F09F0CCC0702F198B088B6D2D8989EA
:105020000E9410278AE593E00E947F23B6C0822F5A
:10503000807F09F047C0651314C0341312C0D1102B
:1050400010C02F70206120935F030E9450278AE5D3
:1050500093E00E947F2380915F03D70115968C9384
:105060002FC00115110519F15F3F11F44F3FF9F001
:10507000CD2CD1101CC0809128032091290336E04B
:10508000821709F45CC090E0389FF001399FF00D61
:105090001124E65DFC4F6181561306C06081461302
:1050A00003C06281611103C001968770E9CFCD2CE6
:1050B000DD2009F426C180915F03816080935F0346
:1050C000C12C1FC1651308C0341306C0D11004C021
:1050D00080915F03D701C9C04D875E87DF86702F3F
:1050E000198B088B6D2D89890E94CB268823E9F1C5
:1050F000DD20D9F120915F03822F82958F7090E09F
:10510000029774F080915A0390915B0398878F8384
:1051100019861B870A872C87CE0107960E947F235A
:1051200086E0F701AAE5B3E001900D928A95E1F7D8
:105130000E945E270E945027CC24C394E2C0702FA7
:10514000198B088B60E089890E94E42B292F229516
:105150002F7030E0223031050CF0C7C09F7009F08D
:10516000C1C0805E883008F4CCC0C7010E947F2394
:10517000E3CF0817190708F456C0F801E81BF90B2C
:10518000CF01883C910508F453C0C12C702F198BB6
:10519000088B6D2D89890E941027EAE5F3E086E0EF
:1051A000DF011D928A95E9F70E945027AAC0651376
:1051B00014C0341312C0D11010C080915F03F701E6
:1051C0008583C7010E947F2386E0EAE5F3E0DF01E3
:1051D0001D928A95E9F7CB2C94C04D875E87DF86B8
:1051E000702F198B088B6D2D89890E94CB268823FF
:1051F00009F4BBCFDD2009F4B8CF20915F03822FE3
:1052000082958F7090E002970CF48ACF80915A03B8
:1052100090915B039A8389831B821D830C832E8369
:10522000CE0101967BCF80959095800F911FA9CFDD
:10523000CD2CDD2009F499CF65132EC034132CC07A
:1052400020915F0320FD1FC0822F82958F70D9F0BF
:10525000D70115962C9315978F3049F08F5F982FB3
:105260009295907F822F8F70892B15968C93C70112
:105270000E947F2386E0F701AAE5B3E001900D923A
:105280008A95E1F791CF86E0F701AAE5B3E00190B6
:105290000D928A95E1F735C04D875E87DF86702FC6
:1052A000198B088B6D2D89890E94CB26811138CFEF
:1052B00080915F03816080935F03C7010E947F2319
:1052C00020C0DD2009F451CF4D875E87DF86702F27
:1052D000198B088B6D2D89890E94CB26882309F4B0
:1052E00044CF1ECF81113DCF0CC0243031050CF0CE
:1052F0003CCF9F7009F435CFF7019581907F09F07D
:1053000030CF8C2D61960FB6F894DEBF0FBECDBFA7
:10531000DF91CF911F910F91FF90EF90DF90CF9091
:10532000BF9008951F93CF93DF93CDB7DEB72C972F
:105330000FB6F894DEBF0FBECDBF4F835887698785
:105340007A878B879C87CE0107960E94B92788238E
:1053500069F08F8198852A853B85232BF1F19F3F4A
:1053600009F063C08F3F09F060C037C086E0FE01DE
:105370003796DE01119601900D928A95E1F76F81C3
:105380007885EA85FB85309741F17F3F11F46F3FC7
:1053900021F12091290330E0C901019687709927F6
:1053A0004091280350E08417950709F447C06983AA
:1053B0007A83FD83EC8396E0929FD001939FB00D9A
:1053C0001124A65DBC4FFE01319601900D929A9575
:1053D000E1F7809329030E942F2716E0809128038C
:1053E000909129038917C1F1189FC0011124865D8E
:1053F0009C4F0E94B927882379F1E09128031E9FD2
:10540000F0011124E65DFC4F40815181628173817E
:10541000848195810E941F278091280390E0019646
:105420008770992780932803D9CF4F815885698544
:105430007A858B859C850E941F27CFCF0E94C72627
:105440001092290310922803EAE5F3E086E0DF01D9
:105450001D928A95E9F7C1CF2C960FB6F894DEBF5E
:105460000FBECDBFDF91CF911F910895DF92EF92D4
:10547000FF920F931F93CF93DF93FC01892B09F4C5
:105480008AC0E12CF12CDD24D394EF012196849184
:10549000853709F461C058F4843708F04EC0843071
:1054A00008F06AC08130D1F0823071F174C0883761
:1054B00009F45DC050F4863709F455C0873709F008
:1054C0006AC08E2D0E949D2C54C09CE7980F903787
:1054D00008F061C08F770E94452350C08F010E5F96
:1054E0001F4FFE01849190E2980F983050F487701E
:1054F000FD2D01C0FF0F8A95EAF78F2F0E94A32C84
:1055000014C00E94E52213C08F010E5F1F4FFE01E1
:10551000C49180E28C0F883060F4C7708D2D01C07B
:10552000880FCA95EAF70E94A92C0E94CA2CE801AC
:1055300025C08C2F0E944523FACF9F012E5F3F4F3D
:10554000FE01C491CC2369F08FE99FE00197F1F748
:1055500000C00000C150F6CF9F012E5F3F4FFE01FB
:10556000F490E9010BC00E948D2CE82E07C00E9428
:10557000A02C0E94CA2C02C00E94E5228F2D8823F5
:1055800041F0EFE9FFE03197F1F700C000008150F2
:10559000F6CFFE017ACFDF91CF911F910F91FF904F
:1055A000EF90DF900895609360047093610480939E
:1055B0006204909363040C94362D08950F931F9307
:1055C0000091640410916504209166043091670491
:1055D000602B712B822B932B609364047093650472
:1055E00080936604909367041F910F910C94352D5E
:1055F0000F931F9300916404109165042091660439
:1056000030916704602371238223932360936404A1
:105610007093650480936604909367041F910F91C3
:105620000C94352D0F931F93009164041091650421
:1056300020916604309167046027712782279327A1
:105640006093640470936504809366049093670488
:105650001F910F910C94352D60E070E0CB010C94FC
:10566000D32A0F931F9341E050E060E070E08A017D
:105670009B0104C0000F111F221F331F8A95D2F710
:10568000C901B8011F910F910C94D32A0F931F9356
:1056900041E050E060E070E004C0440F551F661F19
:1056A000771F8A95D2F78091600490916104A09150
:1056B0006204B09163048A019B01082B192B2A2BE9
:1056C0003B2BC901B8011F910F910C94D32A0F9362
:1056D0001F9341E050E060E070E004C0440F551FAC
:1056E000661F771F8A95D2F7409550956095709503
:1056F0008091600490916104A0916204B091630470
:105700008A019B01082319232A233B23C901B801DD
:105710001F910F910C94D32A0F931F9341E050E0F7
:1057200060E070E004C0440F551F661F771F8A9524
:10573000D2F78091600490916104A0916204B091CD
:1057400063048A019B01082719272A273B27C901DF
:10575000B8011F910F910C94D32A0F931F930091BE
:105760006004109161042091620430916304602B05
:10577000712B822B932B1F910F910C94D32A0F9393
:105780001F93009160041091610420916204309194
:10579000630460237123822393231F910F910C9440
:1057A000D32A0F931F9300916004109161042091FC
:1057B00062043091630460277127822793271F9129
:1057C0000F910C94D32A08958F929F92AF92BF921B
:1057D000DF92EF92FF920F931F93CF93DF9300D04E
:1057E00000D01F92CDB7DEB78A016623C9F1809041
:1057F000640490906504A0906604B0906704809162
:10580000600490916104A0916204B0916304882ABD
:10581000992AAA2ABB2A8FE1E82EF12CD501C401CE
:105820000E2C04C0B695A795979587950A94D2F744
:1058300080FF07C0DE2CB8018E2D0E94742D0197C9
:1058400029F481E0E81AF10848F7D12C80E1189F8B
:10585000F0011124E00FF11DE05AFC4FD08209C085
:1058600080E1189FF0011124E40FF11DE05AFC4F74
:10587000D08009831A8369817A818D2D0E94742DCD
:105880000F900F900F900F900F90DF91CF911F917D
:105890000F91FF90EF90DF90BF90AF909F908F900F
:1058A000089520910B0130910C01F90132969FEF80
:1058B00040E05191581789F09F3F19F4511101C0F0
:1058C000942F4F5F4630A9F79F3F39F0F901E90F58
:1058D000F11D97FDFA9582830895089520910B019B
:1058E00030910C01F9013296285F3F4F9081981357
:1058F00001C010823196E217F307C1F7089581E0E5
:1059000090E0E0910B01F0910C01E80FF91F10827B
:10591000019688309105A9F7089580917204089541
:1059200090917204892B80937204089580959091D0
:1059300072048923809372040895809372040895F9
:1059400010927204089590917104892B80937104D0
:10595000089580959091710489238093710408952E
:105960001092710408958093680408951092680459
:10597000089580910B0190910C01FC0131969C01DE
:10598000285F3F4F80E0919191118F5FE217F307FD
:10599000D1F70895E0910B01F0910C018091720410
:1059A0008083E0910B01F0910C0190818091710452
:1059B000892B808380916804882361F0E0910B013A
:1059C000F0910C019081892B80830E94B92C811168
:1059D0001092680480910B0190910C010C9423218A
:1059E000909399018093980108958295982F9C7CBB
:1059F000392F36953695282F237344E0249FC00114
:105A00001124932F982B292F2A7A2695892F857573
:105A1000880F822B08951F93CF93DF931F92CDB7EA
:105A2000DEB799830E94F52C182F9981892F0E9447
:105A3000F52C212F30E0322F2227A901482BCA0153
:105A40000F90DF91CF911F9108950895CF93DF9329
:105A500000D000D01F92CDB7DEB70F900F900F90FF
:105A60000F900F90DF91CF910895089508950C94B1
:105A7000A2220E94A4220C94C7261F920F920FB656
:105A80000F9211248F939F93AF93BF9380917404CF
:105A9000811113C08091E8029091E902A091EA027D
:105AA000B091EB024196A11DB11D8093E802909345
:105AB000E902A093EA02B093EB02BF91AF919F91EC
:105AC0008F910F900FBE0F901F90189520E1929F1D
:105AD000F0011124E80FF11DE052FF4F9491892F3E
:105AE0008F7092959F700895CF93C82FCB010E941D
:105AF000662D282F30E080E1989FA0011124422BD1
:105B0000532B4038510519F480E090E015C0977090
:105B1000E92FF0E088E0C89FE00DF11D112484E03A
:105B2000EE0FFF1F8A95E1F7E20FF31FEE0FFF1F45
:105B3000E050F84985919491CF91089580E090E0EC
:105B4000089508958091770480FF0BC06091100143
:105B500085E0689FB00111247595679575956795E7
:105B60002BC081FF09C06091100185E0689FB001E2
:105B700011247595679520C082FF07C060911001C0
:105B800085E0689FB001112417C090917804992393
:105B9000D1F060910F01961788F72091100185E0F0
:105BA000289F90011124929FA001939F500D1124D2
:105BB00070E0CA010E94BA316038710540F4611585
:105BC000710539F002C065E070E0862F08958FE717
:105BD000089581E008958091770480FF08C0609166
:105BE0000E0170E0759567957595679521C081FFE9
:105BF00006C060910E0170E07595679519C082FF2F
:105C000004C060910E0170E010C090917804992357
:105C1000C1F060910D019617A0F780910E01899F48
:105C2000C001112470E00E94BA316038710528F477
:105C30006115710521F0862F08958FE7089581E0A1
:105C4000089561E070E0F4CF803F21F40E94A22D1E
:105C5000819504C0813F29F40E94A22D80937B048A
:105C60000895823F21F40E94A22D819504C0833FB4
:105C700029F40E94A22D80937A040895893F19F493
:105C80000E94EB2D05C08A3F31F40E94EB2D8195D7
:105C900080937C0408958B3F21F40E94EB2D819525
:105CA00004C08C3F29F40E94EB2D80937D0408955D
:105CB000843F21F480917904816017C0853F21F4ED
:105CC00080917904826011C0863F21F4809179042B
:105CD00084600BC0873F21F480917904886005C0FF
:105CE000883F31F48091790480618093790408952C
:105CF0008D3F21F48091770481600BC08E3F21F4A9
:105D000080917704826005C08F3F29F480917704E9
:105D10008460809377040895803F39F480917B04F8
:105D200087FF6CC010927B0469C0813F29F4809189
:105D30007B041816BCF362C090917A04823F29F468
:105D400097FF5CC010927A0459C0833F19F419166A
:105D5000CCF354C0893F41F480917C0418160CF0B8
:105D60004DC010927C044AC08A3F29F480917C0483
:105D700087FF44C0F6CF8B3F39F480917D0487FFC5
:105D80003DC010927D043AC08C3F29F480917D047F
:105D90001816BCF333C0843F21F4809179048E7FC0
:105DA00017C0853F21F4809179048D7F11C0863F13
:105DB00021F4809179048B7F0BC0873F21F480917F
:105DC0007904877F05C0883F31F4809179048F7E04
:105DD0008093790413C08D3F21F4809177048E7FE6
:105DE0000BC08E3F21F4809177048D7F05C08F3FDB
:105DF00029F4809177048B7F8093770480917A04D3
:105E000081110EC080917B0481110AC080917C04B5
:105E1000811106C080917D04811102C01092780426
:105E200008958091730483FF7EC082E994E00E940C
:105E3000BD02809179041F928F938DE894E09F9327
:105E40008F930E9456038BE894E00E94BD028091DC
:105E50007A04282F082E000C330B3F938F9388E889
:105E600094E09F938F930E94560386E894E00E94EB
:105E7000BD0280917B04282F082E000C330B3F932A
:105E80008F9383E894E09F938F930E94560381E859
:105E900094E00E94BD0280917C04282F082E000C03
:105EA000330B3F938F938EE794E09F938F930E94E1
:105EB00056038CE794E00E94BD0280917D04282F58
:105EC000082E000C330B3F938F9389E794E09F9348
:105ED0008F930E94560386E794E00E94BD02809152
:105EE00078041F928F9383E794E09F938F930E948F
:105EF000560381E794E00E94BD02809177041F92CF
:105F00008F938EE694E09F938F930E9456038BE6C7
:105F100094E00E94BD028DB79EB74C960FB6F894E0
:105F20009EBF0FBE8DBF89E794E00E946C210E9446
:105F3000200B909376048093750408951F93CF935C
:105F4000DF9380917504909176040E94380BAC0128
:105F500090917804992321F02091110130E006C03E
:105F6000209112018AE0289F9001112442175307C3
:105F700008F485C080917A04C0917B04D0917C04A0
:105F800010917D04811107C0C11175C0D11173C07A
:105F9000111171C074C09F3F19F09F5F90937804F6
:105FA000181624F40E94A22D80937A0480917A041A
:105FB00087FF05C00E94A22D819580937A041C164C
:105FC00024F40E94A22D80937B0480917B0487FFA0
:105FD00005C00E94A22D819580937B0460917A0474
:105FE000662331F1C0917B04CC2311F1062E000C05
:105FF000770B880B990B0E948C3023E333E343E348
:106000005FE30E9441310E94543060937A046C2F08
:10601000CC0F770B880B990B0E948C3023E333E372
:1060200043E35FE30E9441310E94543060937B045C
:106030001D1624F40E94EB2D80937C0480917C0437
:1060400087FF05C00E94EB2D819580937C0411167B
:1060500024F40E94EB2D80937D0480917D0487FFC2
:1060600005C00E94EB2D819580937D04DF91CF9137
:106070001F910C94112F9F3F09F08FCF97CFDF9185
:10608000CF911F910895E9E7F4E085E0DF011D92CB
:106090008A95E9F7109278041092770408950E9487
:1060A000C73008F481E008950E945B306894B11114
:1060B0000C94363108950E941B3188F09F5798F058
:1060C000B92F9927B751B0F0E1F0660F771F881FFD
:1060D000991F1AF0BA95C9F714C0B13091F00E9417
:1060E0003531B1E008950C943531672F782F88272A
:1060F000B85F39F0B93FCCF3869577956795B3953E
:10610000D9F73EF490958095709561957F4F8F4FAC
:106110009F4F0895E89409C097FB3EF490958095B1
:10612000709561957F4F8F4F9F4F9923A9F0F92F5D
:1061300096E9BB279395F695879577956795B795DB
:10614000F111F8CFFAF4BB0F11F460FF1BC06F5FC1
:106150007F4F8F4F9F4F16C0882311F096E911C0D3
:10616000772321F09EE8872F762F05C0662371F0F4
:1061700096E8862F70E060E02AF09A95660F771F08
:10618000881FDAF7880F9695879597F90895990FE4
:106190000008550FAA0BE0E8FEEF16161706E807F1
:1061A000F907C0F012161306E407F50798F0621B12
:1061B000730B840B950B39F40A2661F0232B242BE7
:1061C000252B21F408950A2609F4A140A6958FEF06
:1061D000811D811D089597F99F6780E870E060E058
:1061E00008959FEF80EC089500240A941616170670
:1061F00018060906089500240A94121613061406B8
:1062000005060895092E0394000C11F4882352F01A
:10621000BB0F40F4BF2B11F460FF04C06F5F7F4FD2
:106220008F4F9F4F089557FD9058440F551F59F0B9
:106230005F3F71F04795880F97FB991F61F09F3F73
:1062400079F087950895121613061406551FF2CF9C
:106250004695F1DF08C0161617061806991FF1CFEC
:1062600086957105610508940895E894BB27662713
:106270007727CB0197F908950E94C73008F48FEF74
:1062800008950E9454310C9402310E94F43038F089
:106290000E94FB3020F0952311F00C94EB300C940D
:1062A000F13011240C9436310E94133170F3959F14
:1062B000C1F3950F50E0551F629FF001729FBB27FD
:1062C000F00DB11D639FAA27F00DB11DAA1F649F99
:1062D0006627B00DA11D661F829F2227B00DA11D4C
:1062E000621F739FB00DA11D621F839FA00D611DD2
:1062F000221F749F3327A00D611D231F849F600DF3
:10630000211D822F762F6A2F11249F5750409AF01B
:10631000F1F088234AF0EE0FFF1FBB1F661F771FA7
:10632000881F91505040A9F79E3F510580F00C9472
:10633000EB300C9436315F3FE4F3983ED4F386950E
:1063400077956795B795F795E7959F5FC1F7FE2B12
:10635000880F911D9695879597F90895991B79E077
:1063600004C0991F961708F0961B881F7A95C9F7E5
:106370008095089597FB072E16F4009407D077FDBB
:1063800009D00E94D43107FC05D03EF49095819548
:106390009F4F0895709561957F4F0895EE0FFF1FF1
:1063A0000590F491E02D0994AA1BBB1B51E107C095
:1063B000AA1FBB1FA617B70710F0A61BB70B881F95
:1063C000991F5A95A9F780959095BC01CD01089524
:0463D000F894FFCF6F
:1063D400EB19DC1AB91A851A511A01690428081430
:1063E4000A321E66756C6C006C6F7700000000004A
:1063F400AB090000000021040000000090045F03CA
:10640400AB032204C60361036203C903CE03D303AF
:10641400A203DB03DE03FEFF0000170400000000FC
:10642400410A00000000B00AC319A60AAC0AA90A6E
:10643400AF0AA50A00000000310C870B490C0000CC
:10644400000070165F03CF156019C715BF176203EC
:10645400CA156403404D3622EF03A2036C034A03BA
:08646400D602EF020803210338
:106800008800EA44E944E244040005000600070069
:10681000080009000A000B000C000D000E000F001C
:1068200010001100120013001400150016001700CC
:10683000180019001A001B001C001D001E001F007C
:10684000200021002200230024002500260027002C
:10685000280029002A002B002C002D002E002F00DC
:10686000300031003200330034003500360037008C
:10687000380039003A003B003C003D003E003F003C
:1068800040004100420043004400450046004700EC
:10689000480049004A004B004C004D004E004F009C
:1068A000500051005200530054005500560057004C
:1068B000580059005A005B005C005D005E005F00FC
:1068C00060006100620063006400F1A18500670060
:1068D000680069006A006B006C006D006E006F005C
:1068E0007000710072007300890087008A008B00BD
:1068F000E000E100E200E300E400E500E600E7007C
:106900000100010001000100EA4401000100E2442D
:106910000100010001000100460001004A004B0097
:10692000010001004700480001000100E9440100A6
:106930000100010001000100010001003A003B00DC
:106940003C003D003E003F0040004100420043004B
:10695000010035004C0001000100440045005200D8
:1069600049000100010050004F0029004D004E0079
:1069700051000100010001000100010001000100BF
:1069800001000100010001000100010001000100FF
:1069900001000100010001000100010001004D00A3
:1069A0004A004E004B0001000100010001000100FF
:1069B00001000100010001000100010001000100CF
:1069C00001000100010001000100010001000100BF
:1069D00001000100010001000100010001000100AF
:1069E0000100010001000100490001000100010057
:1069F000010001000100010001000100010001008F
:00000001FF
